:020000001228C4
:080008009600030897000B119C
:100010008C0B0D280D1415088C0017088300960E04
:10002000160E090000308500003086008316D63099
:10003000810010308500C030860083120A309D0098
:100040000A309E0002309F00BD2000308500003045
:100050008600AC2019309500B62086168510051450
:10006000061186141F089B00051E98200D1C3428BD
:100070008D019B0B342886100614051E98200D1C3C
:100080003D288D010616051E98200D1C43288D0164
:10009000061286118616051185151F081D029B0084
:1000A000051E98200D1C50288D019B0B5028851192
:1000B0000515861206161F089B00051E98200D1CAC
:1000C0005D288D019B0B5D280612861586141F087E
:1000D0009B00051E98200D1C69288D019B0B69282B
:1000E000861006100615051085141F081E029B00B9
:1000F000051E98200D1C78288D019B0B78282E2832
:10010000BD200030850000308600AC201430950002
:10011000B62086140616051EA2200D1C8B288D0104
:1001200086100612051EA2200D1C92288D0189281A
:1001300020309C000508EF38EF3C031D00349C0B79
:100140009A28802820309C000508EF38EF3C031DDA
:1001500000349C0BA428242820309C000508EF388C
:10016000FF3C031DAE289C0BAE280800810115083A
:100170008C00A0308B008D0108008B138B1BBD28D9
:100180008B0108000A309A00CB2805309A00CB2852
:1001900001309A00CB287B309900DD309800980B15
:0C01A000CF28990BCD289A0BCB280034F7
:02400E00F93F78
:00000001FF
